:1000000012C019C017C016C015C014C013C012C04A
:1000100011C010C00FC00EC00DC00CC00BC00AC074
:1000200009C008C007C011241FBECFE5D4E0DEBF61
:10003000CDBF87C0E5CF1FB6E0E6F0E079E10CC0A8
:1000400035E13A95D9F040B34470D9F7000000008B
:1000500000000000000000003DD0909A40B390984E
:10006000447041937A9539F035E13A9539F040B3CF
:100070004470D9F3E5CFE0E6F0E03AC030E1371B59
:1000800021F5E0E6F0E031913323F9F4319131913B
:100090003323D9F431913323C1F431913323A9F4BB
:1000A0003191332391F43191332379F43191332316
:1000B000889409F00894E0E6F0E031913081332330
:1000C00011F018F410C008F009C01FBE1895339441
:1000D0001FBE189533E03A95F1F70895EDE1F1E090
:1000E00079E110D0F2CFE6E3F1E071E50BD0EDCF8E
:1000F000662019F4E9E7F0E002C0EAEBF0E071E411
:1001000001D0E5CF3191332369F400008A9A4FE0A2
:100110004A95F1F700008A9842E04A95F1F77A95FE
:1001200089F708958A9A44E04A95F1F700000000A3
:100130008A984CE04A95F1F7000000007A9511F793
:100140000895002407EE05BB00E304BB0FEF08BBD6
:1001500000E007BB0AEF02BB01E001BB02E005BF04
:1001600000E40BBFFAD0C4D0CFD005D1662433242D
:1001700078943320F1F303D000C03324FACFCBEFCF
:10018000D0E001E00992099209920992099209923C
:10019000099209930993CBEFD0E009E0F02EFBD050
:1001A000FF2049F00895662019F4CAEBD0E00895C5
:1001B000C9E7D0E00895ABEFB0E0F5DF0D910F8314
:1001C0000D910E830D9109870D910B830D910C8775
:1001D0000D910D870D910F870D910E8712960D9140
:1001E0000B870D910A870985FF24002309F0F094FD
:1001F00018E0E096F9921A95E9F7D5DF0A85FF2411
:10020000002309F0F09418E0E896F9921A95E9F7BE
:10021000ABEFB0E0C8DF1C960D91002329F40D91DF
:10022000002321F40FE703C00FEF01C000E010E846
:10023000A896F12EF022F9921695D9F7ABEFB0E01F
:10024000B2DF1E960D91002329F40D91002321F4B5
:100250000FE703C000E001C00FEF10E8A096F12EF9
:10026000F022F9921695D9F7ABEFB0E0509610E86E
:1002700022270D91002309F0212B1695D1F71FE7B6
:10028000210F91DF609610E8F12EF222F992169577
:10029000D9F7ABEFB0E0589610E822270D91002374
:1002A00009F0212B1695D1F71FE7210F7CDF689607
:1002B00010E8F12EF222F9921695D9F7609408957C
:1002C0000EE10A95F1F708951F9317E60FEF00006E
:1002D0000000000000000000000000000A95B9F7CF
:1002E00000000000000000001A9581F71F9108959A
:1002F00031E0EDE1F1E034963083339630833B9684
:10030000308336963083089531E0E6E3F1E03896A5
:1003100030833896308336963193308332963193DA
:1003200031933193308332963083329630833796CF
:1003300030833296319331933193319331933083BB
:1003400035963083329631933083359630833396A9
:10035000319330837196308308954427EDE1F1E0C5
:1003600039E141933A95E9F7E6E3F1E031E541936C
:100370003A95E9F70895AAEBB0E0E9E7F0E0C6E3C3
:10038000D1E000E4499141934D930A95D9F741E0BA
:1003900041934D9308950991002369F40000A39AB5
:1003A0001FE01A95F1F70000A39812E01A95F1F7F3
:1003B000FA9489F70EC0A39A14E01A95F1F7000099
:1003C0000000A3981CE01A95F1F700000000FA94D1
:1003D00011F7CBEFD0E021E205E10A95F1F013B37C
:1003E0001870D9F7000000000000000000000000B5
:1003F00010D0909A13B39098187019932A9539F0E9
:1004000005E10A9551F013B31870D9F3E5CFFF2435
:10041000089503E00A95F1F70895FF24F3940895F1
:00000001FF
